:10000000B6010929A501A400B7172730A3001030B5
:1000100015200330A300E8301520A301643015201B
:10002000A3010A30152024082028A2002508A100D9
:100030002408A000D2202008031DB713B71B080016
:10004000303EA7000711871007108316071187108D
:100050000710F030860583122708B6184D283A306D
:10006000A1009830AA203330A60062201330A100EE
:100070008830AA2062206430A92062206430A92040
:100080002230A600622028304C200C304C20063054
:100090004C20B61427084D283614A600361C5B28C1
:1000A0008710033C031C602860200730A100D0307B
:1000B000AA20031408003614FE3C031904298714EF
:1000C000A60E361C36100715F030860526080F39A7
:1000D00086040711A60E361862283230A9200314B0
:1000E0000800A000A00DA00DA00D3830A0058130A3
:1000F00020049F000030A1003230AA201F151F19D4
:100100007F281E08A10083161E08042903178D00EE
:1001100083168C130C1483120C08042903178C000B
:1001200083168C130C1555308D00AA308D008C145D
:100130008C1898280C110429A301A200FF30A207F3
:10014000031CA307031C04290330A100E730AA20E5
:100150009E28A101FC3EA000A109031CB528FF3088
:100160000000A0070318B028A0076400A10FAF2863
:100170000800A2000330C228A2000130C228A20059
:100180000430C228A80023082102031DC928220820
:100190002002043003180130031902302805031D22
:1001A000FF3004291030A600A501A401210DA40DE3
:1001B000A50D2208A4022308031C230FA50203187F
:1001C000E8282208A40723080318230FA507031013
:1001D000A00DA10DA60BD628200804291030A800D8
:1001E000A101A001A70CA60C031CFC282208A00753
:1001F00023080318230FA107A10CA00CA50CA40C25
:10020000A80BF22824080429831303138312640023
:1002100008008316DF30850082309F007030860032
:100220008113870183128501860187018A11B8290C
:10023000861783168613FE3083128A01212001302F
:100240008A01212050308A01212069308A01212031
:1002500074308A01212020308A01212043308A0114
:1002600021206F308A0121206D308A0121207030D9
:100270008A01212020308A01212052308A01212048
:1002800065308A01212076308A01212030308A01B0
:1002900021202E308A01212031308A012120033093
:1002A000A300E8308A019D20FE308A012120C03061
:1002B0008A01212050308A01212072308A012120B8
:1002C0006F308A01212064308A01212075308A0133
:1002D000212063308A01212065308A012120643089
:1002E0008A01212020308A01212062308A012120C8
:1002F00079308A01212020308A01212041308A0171
:1003000021204F308A01212052308A012120633080
:100310008A0121200330A300E8308A019D200800D3
:1003200003308A017120BC002108BD000A308A0117
:100330009C20080002308A017120C2002108C300FD
:100340000A308A019C20080001308A017120C60011
:100350002108C7000A308A019C20080000308A0169
:100360007120CA002108CB000A308A019C200800B5
:1003700007138316071383120712831607128312BB
:1003800087118316871183128512831685128312B3
:100390008A0118213E30E8003E30E9003E30EA0094
:1003A0003E30EB0064308A019C2064008A11061FF5
:1003B000D229861383168613FE3083128A012120E8
:1003C00001308A01212042308A0121203A308A01FD
:1003D000212048308A01212065308A0121206130A6
:1003E0008A01212074308A01212020308A012120B5
:1003F00063308A0121206F308A0121206E308A010A
:10040000212074308A01212072308A0121206F302E
:100410008A0121206C308A012120FE308A012120AE
:10042000C0308A01212059308A0121203A308A01C6
:1004300021204D308A0121206F308A012120743023
:100440008A0121206F308A01212072308A01212007
:1004500020308A01212064308A01212072308A01F3
:10046000212065308A01212073308A0121207330D8
:100470008A0121200130A3002C308A019D206400D4
:100480008A11061E492A64008A15861E812D8A015A
:100490003F2A64308A019C2064008A11061E492A82
:1004A000861383168613FE3083128A0121200130C1
:1004B0008A01212042308A0121203A308A012120FC
:1004C00054308A01212069308A01212072308A014A
:1004D000212065308A01212020308A0121206330CB
:1004E0008A0121206F308A0121206E308A0121206B
:1004F00074308A01212072308A0121206F308A01F4
:1005000021206C308A012120FE308A012120C03058
:100510008A01212059308A0121203A308A01212084
:1005200042308A01212061308A01212074308A0101
:10053000212074308A01212065308A012120723007
:100540008A01212079308A01212020308A0121204E
:1005500063308A0121206F308A0121206E308A01A8
:10056000212074308A01212072308A0121206F30CD
:100570008A0121206C308A0121200130A3002C3017
:100580008A019D2064008A11061EC92F64008A1109
:10059000861ECC2A8A01C22A64308A019C2064000B
:1005A0008A11861ECC2A0C308A018620D600D701FB
:1005B0000D308A018620D800D9010E308A018620AC
:1005C000DA00DB010D308A018620DC00DD01FE301F
:1005D0008A01212001308A01212054308A01212002
:1005E00065308A0121206D308A01212070308A0116
:1005F00021205708A50056088A0103203A308A01B5
:1006000021205908A50058088A0103203A308A01A0
:1006100021205B08A5005A088A0103203A308A018C
:1006200021205D08A5005C088A010320FE308A01B4
:100630002120C0308A01212043308A0121206830E6
:100640008A01212061308A0121206E308A01212017
:1006500067308A01212065308A0121203F308A01DC
:10066000212020308A01212052308A0121203A3075
:100670008A0121204E308A01212020308A01212048
:1006800042308A0121203A308A01212059308A01E2
:100690002120C8308A019C2064008A11061E562B36
:1006A00064008A11061FEE2D8A154B2864308A01DA
:1006B0009C2064008A11061E562BFE308A012120E0
:1006C00001308A01212042308A01212020308A0114
:1006D000212042308A01212061308A01212074309A
:1006E0008A01212074308A01212020308A012120B2
:1006F00054308A01212065308A0121206D308A0121
:10070000212070308A0121203D308A0121205708A4
:10071000A50056088A010320FE308A012120C0303E
:100720008A01212052308A0121203A308A01212079
:100730004E308A01212065308A01212078308A01DB
:10074000212074308A01212020308A012120593053
:100750008A0121203A308A01212044308A01212057
:100760006E308A01212020308A01212042308A0106
:1007700021203A308A01212055308A012120703011
:100780008A012120C8308A019C2064008A11061E3B
:10079000D32B64008A11861EE62B64008A11061F83
:1007A000FC2B8A01C52BD60A0319D70A5608A000CC
:1007B0005708A100A3013C308A01BF208A11031D04
:1007C000E42B3C30D600D7018A01562B0130D602EB
:1007D0000030031C013ED7025608A0005708A100B4
:1007E000A3010A308A01BC208A11031DFA2B0A30AA
:1007F000D600D7018A01562B64308A019C20640000
:100800008A11061FFC2BFE308A01212001308A014B
:10081000212042308A01212020308A0121204230CB
:100820008A01212061308A01212074308A0121202F
:1008300074308A01212020308A01212054308A011D
:10084000212065308A0121206D308A0121207030FD
:100850008A0121203D308A0121205908A50058082D
:100860008A010320FE308A012120C0308A01212024
:1008700052308A0121203A308A0121204E308A01EB
:10088000212065308A01212078308A0121207430AE
:100890008A01212020308A01212059308A0121201B
:1008A0003A308A01212044308A0121206E308A01A9
:1008B000212020308A01212042308A0121203A3033
:1008C0008A01212055308A01212070308A0121209F
:1008D000C8308A019C2064008A11061E792C6400AD
:1008E0008A11861E8C2C64008A11061FA22C8A0194
:1008F0006B2CD80A0319D90A5808A0005908A1007E
:10090000A3013C308A01BF208A11031D8A2C3C3090
:10091000D800D9018A01FC2B0130D8020030031C19
:10092000013ED9025808A0005908A100A3010A30CD
:100930008A01BC208A11031DA02C0A30D800D901DD
:100940008A01FC2B64308A019C2064008A11061FF6
:10095000A22CFE308A01212001308A012120423060
:100960008A01212020308A01212042308A01212061
:1009700061308A01212074308A01212074308A017B
:10098000212020308A01212054308A012120653025
:100990008A0121206D308A01212070308A012120B6
:1009A0003D308A0121205B08A5005A088A010320F6
:1009B000FE308A012120C0308A01212052308A0174
:1009C00021203A308A0121204E308A0121206530D1
:1009D0008A01212078308A01212074308A01212067
:1009E00020308A01212059308A0121203A308A01A1
:1009F000212044308A0121206E308A0121202030BC
:100A00008A01212042308A0121203A308A012120A6
:100A100055308A01212070308A012120C8308A0196
:100A20009C2064008A11061E1F2D64008A11861EF8
:100A3000322D64008A11061F482D8A01112DDA0A11
:100A40000319DB0A5A08A0005B08A100A3013C308F
:100A50008A01BF208A11031D302D3C30DA00DB01F2
:100A60008A01A22C0130DA020030031C013EDB02B5
:100A70005A08A0005B08A100A3010A308A01BC202B
:100A80008A11031D462D0A30DA00DB018A01A22CEF
:100A900064308A019C2064008A11061F482DFE30B4
:100AA0008A01212001308A01212042308A0121203F
:100AB00020308A01212042308A01212061308A01C0
:100AC000212074308A01212074308A0121202030B5
:100AD0008A01212054308A01212065308A01212099
:100AE0006D308A01212070308A0121203D308A0139
:100AF00021205D08A5005C088A010320FE308A01E0
:100B00002120C0308A01212052308A0121203A3030
:100B10008A0121204E308A01212065308A0121205E
:100B200078308A01212074308A01212020308A0106
:100B3000212059308A0121203A308A012120443075
:100B40008A0121206E308A01212020308A01212053
:100B500042308A0121203A308A01212055308A0111
:100B6000212070308A012120C8308A019C20640035
:100B70008A11061EC52D64008A11861ED82D6400B8
:100B80008A11061FEE2D8A01B72DDC0A0319DD0A32
:100B90005C08A0005D08A100A3013C308A01BF20D1
:100BA0008A11031DD62D3C30DC00DD018A01482D61
:100BB0000130DC020030031C013EDD025C08A000B5
:100BC0005D08A100A3010A308A01BC208A11031D1F
:100BD000EC2D0A30DC00DD018A01482D8A019021CC
:100BE0003C08A6003D08A7007D30A200A3018A01B1
:100BF000EE20B2002508B3003208A0003308A1009F
:100C0000A2010130A3008A01D220BE002108BF004A
:100C10008A019A214208A6004308A7007D30A2005D
:100C2000A3018A01EE20B2002508B3003208A0001B
:100C30003308A100A2010130A3008A01D220C40020
:100C40002108C5008A01A4214608A6004708A7007C
:100C50007D30A200A3018A01EE20B2002508B30076
:100C60003208A0003308A100A2010130A3008A01CC
:100C7000D220C8002108C9008A01AE214A08A60076
:100C80004B08A7007D30A200A3018A01EE20B2002C
:100C90002508B3003208A0003308A100A2010130EA
:100CA000A3008A01D220CC002108CD00FE308A01A9
:100CB000212001308A01212041308A01212057085A
:100CC000A50056088A0103203A308A0121204230CB
:100CD0008A0121205908A50058088A0103203A30CA
:100CE0008A01212043308A0121205B08A5005A088F
:100CF0008A0103203A308A01212044308A012120D0
:100D00005D08A5005C088A01032020308A012120AB
:100D100020308A012120FE308A012120C0308A0142
:100D2000212068088A0121203F08A5003E088A0189
:100D3000032020308A012120FE308A012120C0308A
:100D40008A012120FE308A01212014308A012120CD
:100D5000FE308A01212014308A012120FE308A01D0
:100D6000212014308A0121203A308A01212069088B
:100D70008A0121204508A50044088A01032020306B
:100D80008A012120FE308A012120C0308A012120E1
:100D9000FE308A01212014308A012120FE308A0190
:100DA000212014308A012120FE308A0121201430B4
:100DB0008A012120FE308A01212014308A0121205D
:100DC000FE308A01212014308A012120FE308A0160
:100DD000212014308A012120FE308A012120143084
:100DE0008A0121203A308A0121206A088A012120C3
:100DF0004908A50048088A01032020308A012120E3
:100E0000FE308A012120C0308A012120FE308A0173
:100E1000212014308A012120FE308A012120143043
:100E20008A012120FE308A01212014308A012120EC
:100E3000FE308A01212014308A012120FE308A01EF
:100E4000212014308A012120FE308A012120143013
:100E50008A012120FE308A01212014308A012120BC
:100E6000FE308A01212014308A012120FE308A01BF
:100E7000212014308A012120FE308A0121201430E3
:100E80008A012120FE308A01212014308A0121208C
:100E90003A308A0121206B088A0121204D08A500E3
:100EA0004C088A01032020308A01212064008A1125
:100EB000061FB8293E08A0003F08A1005708A3005C
:100EC00056088A01BF208A11031D6E2F071383164F
:100ED000071383122D30E8008A11742F0717831629
:100EE000071383122B30E8004408A0004508A10036
:100EF0005908A30058088A01BF208A11031D882FB2
:100F000007128316071283122D30E9008A118E2FE3
:100F100007168316071283122B30E9004808A00039
:100F20004908A1005B08A3005A088A01BF208A1162
:100F3000031DA22F87118316871183122D30EA001B
:100F40008A11A82F87158316871183122B30EA0088
:100F50004C08A0004D08A1005D08A3005C088A01B0
:100F6000BF208A11031DBC2F8512831685128312A0
:100F70002D30EB008A11C22F85168316851283123D
:100F80002B30EB000330A300CA308A019D208A0178
:100F9000EE2D64308A019C2064008A11061EC92F40
:100FA00005308A018620E400E50109308A018620A7
:100FB000DE00DF010A308A018620E000E1010B300B
:100FC0008A018620E200E301E601E701FE308A01A2
:100FD000212001308A01212054308A0121206530EE
:100FE0008A0121206D308A01212070308A01212060
:100FF0006508A50064088A0103203A308A0121208F
:101000005F08A5005E088A0103203A308A0121208A
:101010006108A50060088A0103203A308A01212076
:101020006308A50062088A010320FE308A0121209E
:10103000C0308A01212043308A01212068308A0192
:10104000212061308A0121206E308A012120673001
:101050008A01212065308A0121203F308A01212028
:1010600020308A01212052308A0121203A308A0121
:1010700021204E308A01212020308A012120423057
:101080008A0121203A308A01212059308A01212009
:10109000C8308A019C2064008A15061E5528640009
:1010A0008A15061FE72A8A154B2864308A019C207E
:1010B00064008A15061E5528FE308A012120013061
:1010C0008A01212041308A01212020308A012120FB
:1010D00054308A01212065308A0121206D308A0137
:1010E000212070308A0121202E308A0121202030D9
:1010F0008A01212073308A01212065308A01212054
:1011000074308A0121203D308A0121206508A50024
:1011100064088A010320FE308A012120C0308A0140
:10112000212052308A0121203A308A0121204E307C
:101130008A01212065308A01212078308A0121200E
:1011400074308A01212020308A01212059308A01FF
:1011500021203A308A01212044308A0121206E303A
:101160008A01212020308A01212042308A01212059
:101170003A308A01212055308A01212070308A01BD
:101180002120C8308A019C2064008A15061ED228BE
:1011900064008A15861EE52864008A15061FFB2850
:1011A0008A15C428E40A0319E50A6408A000650842
:1011B000A100A30150308A01BF208A15031DE32836
:1011C0005030E400E5018A155C280130E40200306B
:1011D000031C013EE5026408A0006508A100A3010C
:1011E0000A308A01BC208A15031DF9280A30E40060
:1011F000E5018A155C2832308A019C2064008A153A
:10120000061FFB28FE308A01212001308A0121209F
:1012100042308A01212020308A01212054308A0165
:10122000212065308A0121206D308A012120703013
:101230008A0121202E308A01212020308A0121209C
:1012400073308A01212065308A01212074308A019F
:1012500021203D308A0121205F08A5005E088A0117
:101260000320FE308A012120C0308A012120523023
:101270008A0121203A308A0121204E308A01212022
:1012800065308A01212078308A01212074308A015A
:10129000212020308A01212059308A0121203A3032
:1012A0008A01212044308A0121206E308A012120C8
:1012B00020308A01212042308A0121203A308A01DF
:1012C000212055308A01212070308A012120C83028
:1012D0008A019C2064008A15061E782964008A15FC
:1012E000861E8B2964008A15061FA1298A156A2982
:1012F000DE0A0319DF0A5E08A0005F08A100A3014F
:1013000050308A01BF208A15031D89295030DE0024
:10131000DF018A1502290130DE020030031C013E84
:10132000DF025E08A0005F08A100A3010A308A0165
:10133000BC208A15031D9F290A30DE00DF018A15B3
:10134000022932308A019C2064008A15061FA129D7
:10135000FE308A01212001308A01212043308A0198
:10136000212020308A01212054308A01212065303B
:101370008A0121206D308A01212070308A012120CC
:101380002E308A01212020308A01212073308A01E9
:10139000212065308A01212074308A0121203D30CE
:1013A0008A0121206108A50060088A010320FE301F
:1013B0008A012120C0308A01212052308A01212057
:1013C0003A308A0121204E308A01212065308A017D
:1013D000212078308A01212074308A012120203098
:1013E0008A01212059308A0121203A308A012120A6
:1013F00044308A0121206E308A01212020308A0168
:10140000212042308A0121203A308A0121205530A2
:101410008A01212070308A012120C8308A019C2055
:1014200064008A15061E1E2A64008A15861E312A4B
:1014300064008A15061F472A8A15102AE00A031934
:10144000E10A6008A0006108A100A30150308A01F0
:10145000BF208A15031D2F2A5030E000E1018A15B4
:10146000A8290130E0020030031C013EE1026008BF
:10147000A0006108A100A3010A308A01BC208A15DE
:10148000031D452A0A30E000E1018A15A8293230FF
:101490008A019C2064008A15061F472AFE308A01B3
:1014A000212001308A01212044308A01212020306E
:1014B0008A01212054308A01212065308A012120AF
:1014C0006D308A01212070308A0121202E308A015E
:1014D000212020308A01212073308A0121206530AB
:1014E0008A01212074308A0121203D308A01212087
:1014F0006308A50062088A010320FE308A012120CA
:10150000C0308A01212052308A0121203A308A01DC
:10151000212047308A0121206F308A01212020308C
:101520008A01212059308A0121203A308A01212064
:1015300044308A0121206E308A01212020308A0126
:10154000212042308A0121203A308A012120553061
:101550008A01212070308A012120C8308A019C2014
:1015600064008A15061EBE2A64008A15861ED12ACA
:1015700064008A15061FE72A8A15B02AE20A0319B1
:10158000E30A6208A0006308A100A30150308A01A9
:10159000BF208A15031DCF2A5030E200E3018A15CF
:1015A0004E2A0130E2020030031C013EE3026208D1
:1015B000A0006308A100A3010A308A01BC208A159B
:1015C000031DE52A0A30E200E3018A154E2A643041
:1015D0008A019C2064008A15061FE72A031705303C
:1015E0008D00031364088A018E20031709308D00D3
:1015F00003135E088A018E2003170A308D0003133F
:1016000060088A018E2003170B308D0003136208D7
:101610008A018E200713831607138312071283167D
:10162000071283128711831687118312851283167E
:1016300085128312E60A0319E70A6608A000670804
:10164000A1000E30A30010308A01BC208A15031DB2
:10165000042D8A0190213C08A6003D08A7007D309A
:10166000A200A3018A01EE20B2002508B3003208CF
:10167000A0003308A100A2010130A3008A01D220FA
:10168000BE002108BF008A019A214208A600430833
:10169000A7007D30A200A3018A01EE20B200250838
:1016A000B3003208A0003308A100A2010130A3005A
:1016B0008A01D220C4002108C5008A01A42146085D
:1016C000A6004708A7007D30A200A3018A01EE20F2
:1016D000B2002508B3003208A0003308A100A2011F
:1016E0000130A3008A01D220C8002108C9008A0164
:1016F000AE214A08A6004B08A7007D30A200A30136
:101700008A01EE20B2002508B3003208A000330899
:10171000A100A2010130A3008A01D220CC0021083F
:10172000CD00FE308A01212001308A012120413084
:101730008A0121206508A50064088A0103203A3047
:101740008A01212042308A0121205F08A5005E081D
:101750008A0103203A308A01212043308A01212066
:101760006108A50060088A0103203A308A0121201F
:1017700044308A0121206308A50062088A01032001
:1017800020308A01212020308A012120FE308A0168
:101790002120C0308A01212068088A0121203F08C9
:1017A000A5003E088A01032020308A012120FE3056
:1017B0008A012120C0308A012120FE308A012120A7
:1017C00014308A012120FE308A01212014308A0140
:1017D0002120FE308A01212014308A0121203A3054
:1017E0008A01212069088A0121204508A5004408B2
:1017F0008A01032020308A012120FE308A01212025
:10180000C0308A012120FE308A01212014308A0153
:101810002120FE308A01212014308A012120FE304F
:101820008A01212014308A012120FE308A012120E2
:1018300014308A012120FE308A01212014308A01CF
:101840002120FE308A01212014308A012120FE301F
:101850008A01212014308A0121203A308A01212076
:101860006A088A0121204908A50048088A01032046
:1018700020308A012120FE308A012120C0308A01D7
:101880002120FE308A01212014308A012120FE30DF
:101890008A01212014308A012120FE308A01212072
:1018A00014308A012120FE308A01212014308A015F
:1018B0002120FE308A01212014308A012120FE30AF
:1018C0008A01212014308A012120FE308A01212042
:1018D00014308A012120FE308A01212014308A012F
:1018E0002120FE308A01212014308A012120FE307F
:1018F0008A01212014308A012120FE308A01212012
:1019000014308A0121203A308A0121206B088A0193
:1019100021204D08A5004C088A01032020308A01AF
:10192000212064008A11061FB8293E08A0003F0844
:10193000A1006508A30064088A01BF208A15031D61
:10194000A92C07138316071383122D30E8008A157C
:10195000AF2C07178316071383122B30E8004408B7
:10196000A0004508A1005F08A3005E088A01BF200F
:101970008A15031DC32C07128316071283122D30FC
:10198000E9008A15C92C07168316071283122B301B
:10199000E9004808A0004908A1006108A300600808
:1019A0008A01BF208A15031DDD2C8711831687113C
:1019B00083122D30EA008A15E32C871583168711D0
:1019C00083122B30EA004C08A0004D08A1006308E8
:1019D000A30062088A01BF208A15031DF72C851217
:1019E0008316851283122D30EB008A15FD2C851687
:1019F0008316851283122B30EB000330A300CA300C
:101A00008A019D208A151A2B071383160713831248
:101A10000712831607128312871183168711831208
:101A2000851283168512FE3083128A01212001302F
:101A30008A0121204F308A01212076308A0121201D
:101A400065308A01212072308A01212020308A01EC
:101A5000212031308A01212020308A012120683064
:101A60008A0121206F308A01212075308A012120CE
:101A700072308A01212020308A01212021308A0100
:101A80002120FE308A012120C0308A0121204830E7
:101A90008A01212065308A01212061308A012120BC
:101AA00074308A01212020308A0121206F308A0180
:101AB000212066308A01212066308A0121202030D1
:101AC0008A01212062308A01212079308A01212077
:101AD00020308A01212074308A01212069308A0156
:101AE00021206D308A01212065308A012120861352
:101AF00083168613831264008A11061FB8298A157B
:101B00007B2D64308A019C2064008A15861E812DFD
:101B1000861383168613063083128A018620ED0011
:101B200009308A018620EC0064308A019C20640020
:101B30008A15061F942DFE308A01212001308A016A
:101B4000212054308A01212069308A0121206D3002
:101B50008A01212065308A01212072308A012120EA
:101B60003D308A0121206D088A01022030308A012F
:101B7000212073308A01212065308A0121206330C1
:101B80008A012120FE308A012120C0308A012120D3
:101B900052308A0121203A308A0121204E308A01B8
:101BA000212065308A01212078308A01212074307B
:101BB0008A01212020308A01212059308A012120E8
:101BC0003A308A01212044308A0121206E308A0176
:101BD000212020308A01212042308A0121203A3000
:101BE0008A01212055308A01212070308A0121206C
:101BF00096308A019C2064008A15061E092E640016
:101C00008A15861E142E64008A15061F1F2E8A153B
:101C1000FB2DED0A6400FA306D028A15031C122EAA
:101C2000FA30ED008A159B2DED03640002306D0241
:101C30008A1503181D2E0130ED008A159B2D643086
:101C40008A019C2064008A15061F1F2EFE308A011F
:101C5000212001308A01212044308A012120753061
:101C60008A01212074308A01212079308A012120C3
:101C70003D308A0121206C088A01022025308A012A
:101C80002120FE308A012120C0308A0121205230DB
:101C90008A0121203A308A01212053308A012120F3
:101CA00074308A01212020308A01212059308A0194
:101CB00021203A308A01212044308A0121206E30CF
:101CC0008A01212020308A01212042308A012120EE
:101CD0003A308A01212055308A01212070308A0152
:101CE000212096308A019C2064008A15061E822ECF
:101CF00064008A15861E8D2E64008A15061F982E94
:101D00008A15742EEC0A640046306C028A15031C96
:101D10008B2E4630EC008A15262EEC03640003302F
:101D20006C028A150318962E0230EC008A15262EB6
:101D3000031706308D0003136D088A018E200317E8
:101D400009308D0003136C088A018E2086178316D4
:101D500086138312D201D3015208A0005308A100B8
:101D6000B630A3006C308A01BC208A15031DDF2E1B
:101D7000071783160713031083126C0DB200B3010B
:101D8000B30D3308A10032088A01AA200713831675
:101D9000071383126C08643CB2000030031CFF3E42
:101DA000B3000310B20DB30D3308A10032088A014D
:101DB000AA20D20A0319D30A8A15031DAC2E0330B8
:101DC0008A017120BC002108BD003C08A6003D0826
:101DD000A7007D30A200A3018A01EE20B2002508F1
:101DE000B3003208A0003308A100A2010130A30013
:101DF0008A01D220BE002108BF00ED03FE308A0117
:101E00002120C0308A01212052308A0121206530F2
:101E10008A0121206D308A01212061308A01212030
:101E200069308A0121206E308A0121206D088A01E3
:101E3000022030308A01212073308A0121203A307B
:101E40008A0121203F08A5003E088A010320633053
:101E50008A01212020308A01212020308A0121207E
:101E600020308A01212020308A01212020308A015F
:101E7000212064008A11061FB82964006D08003C07
:101E80008A150319512F3E08A0003F08A100410800
:101E9000A30040088A01B9208A15031D792F8A15ED
:101EA000AA2E07138316071383128613831686132D
:101EB000FE3083128A01212001308A012120463020
:101EC0008A01212069308A0121206E308A01212077
:101ED00069308A01212073308A01212068308A010B
:101EE000212020308A01212021308A0121208A15D9
:101EF0007B2D861383168613FE3083128A012120E0
:101F000001308A0121204F308A01212076308A0158
:101F1000212065308A01212072308A012120203061
:101F20008A01212074308A01212065308A01212014
:101F30006D308A01212070308A0121202E308A01E3
:101F4000212021308A0121208A157B2D63008A15EA
:021F5000A62FBA
:02400E00723D01
:10420A001E001200000032001E001E001E002800C0
:06421A0028002800280026
:00000001FF
